:100000002828A301A200FF30A207031CA307031C9A
:1000100023280330A100DF300F200328A101E83E90
:10002000A000A109FC30031C1828A00703181528FC
:10003000A0076400A10F152820181E28A01C222844
:1000400000002228080083130313831264000800B1
:100050008501073099008316850183128B010B11EE
:1000600083168730810083120510831605108312D2
:100070008514831685108514831281016400333042
:100080000102031C442849286400851C48283E2896
:1000900034280514831605108312851083168510E5
:1000A00083120130A30090300220342863005628C8
:02400E00C43FAD
:00000001FF
